:03000000020323D5
:100030007E107F00DFFEDEFC227E067F00DFFEDE1C
:10004000FC22C291900000D291A320B6FCC2912262
:10005000E8C2B5A2E092B2A2E192B3A2E292B422C7
:10006000A2E79297A2E69296A2E59295A2E49294D4
:10007000000000D293000000C29322C2928002D2FC
:1000800092FD1160EDC4116020920211397E64DE90
:10009000FE2275900111307590211170113074019C
:1000A000117B740C117B7428117B7440117B9003BD
:1000B000FB11BE7480117B227402117B1130E4931A
:1000C0006005A3117F80F722C0E0C411D2D0E011F7
:1000D000D222540F240383117F223031323334353E
:1000E00036373839414243444546C0E0E5F011C84F
:1000F000D0E00200C8F5F030E70A742D117FE5F07A
:10010000F40480067420117FE5F075F064842430D7
:10011000117FE5F075F00A842430117FE5F024307A
:10012000117F22C2D57C107D27315E7CE87D0331B2
:100130005E31737C647D00315E20D5086006FC74FE
:1001400020117FEC3173EA75F00A842430117F208E
:10015000D50B742C117FE5F0243012007F2278003B
:1001600008C3EA9CFAEB9DFB50F618EA2CFAEB3D2B
:10017000FBE8226007D2D5243002007F20D5F82288
:100180003098FDC298E599223099FDF599C29922DF
:10019000C0E0E493600CA2E7547F1201884003A3FF
:1001A00080F0D0E0227A08FBC3942940027B28EB40
:1001B000602F1AB401067400117F8025B402067402
:1001C00001117F801CB403067402117F8013B404F4
:1001D000067403117F800AC39405FB74FF117F80AE
:1001E000CEEA6006742E117FDAFA2285F009F5084E
:1001F0008AF0A4F50C85F00DE5098BF0A4F50E85C9
:10020000F00FE5098AF0A4250DF50DE5F0350EF5A2
:100210000EE4350FF50FE5088BF0A4250DF50DE57F
:10022000F0350EF50EE4350FF50F227C007D007ED3
:1002300001E582458370057B037AE722E58320E7A9
:1002400019E582C333F582E58333F5830E80EDC370
:10025000E58313F583E58213F582EAC39582F9EB12
:1002600095834003FBAA01B3EC33FCED33FDDEDFE5
:10027000AB05AA04228583F0E582AB83AA8231EB29
:10028000E50FC313F50FE50E13F50EE50D13F50D90
:10029000E50FA2E0E50E13FBE50D13FA22E57EC3A0
:1002A000357CFAE57F357DFB75F000740A31EBABE8
:1002B0000DAA0CE57EC3957CF582E57F957DF583DF
:1002C0005006758200758300512BBB03054009BAA7
:1002D000E70040047B037AE722AB7DAA7C75F0003F
:1002E000742831EBAB0DAA0C857F83857E82512B60
:1002F000EA225357522D4D65746572204F562044A3
:10030000313100627920444C374A47522020323044
:10031000303120004657443A005245563A00535770
:10032000523A00758122D292C294C295C296C29767
:10033000C293C291758DFD438700758921759852CE
:1003400043885075A88075B800790A1130D9FC111E
:100350009211309002F211B874C0117B9003031116
:10036000BE79C81130D9FC74CF117B742D117F7800
:10037000081818115011301142E58254F845837065
:100380000BE870ED79141130D9FC6167887974CF6E
:10039000117BE8C3132441117F74C0117B900314B7
:1003A00011BEA8790811501130114285827C8583D5
:1003B0007DA879115011301142E58254F8458360CF
:1003C000A685827E85837F517531237420117F90AD
:1003D000031911BE857C82857D835175312390037D
:1003E0001E11B8519D8A7A8B7B31237420117F5165
:1003F000D931A579141130D9FC61999090909090E1
:1004000090909098989898989898989C9C9C9C9C70
:0C0410009C9C9C9E9E9E9E9E9E9E9E001C
:00000001FF
